:1000000000000000000008280000000000000000C0
:10001000283084005830A0008001840AA00B0C28EE
:10002000103095002730960000308E0000308F0091
:10003000013090000B30970007309F008316FF308F
:10004000850083128316CF30860083120C1D26286C
:100050000C116400A914A9182915A91C2911A911AA
:1000600029192916291D2912851B37282912291E0D
:100070003A28A91529192916291D2912051B4128D5
:100080002912291E4428A915A9192915A91D2911C4
:100090002919A916291DA912291F4F282911A91AA2
:1000A0002917A91E2913291D5A28A91B5A28AA0F46
:1000B0005A28AB0A2919A917291DA91300302B02A8
:1000C00003196928A00020092B05A006A01B6E2893
:1000D000702801302A02031C6E287028291171280B
:1000E000291529198616291D8612A9182915A91C52
:1000F0002911861A7C282911291D932827302D02C1
:1001000003198928A00020092D05A006A01B8E2810
:1001100092280F302C02031C8E289228AC0F9128B5
:10012000AD0A291197280030AC000030AD00291D20
:10013000AE2827302F020319A428A00020092F057C
:10014000A006A01BA928AD280F302E02031CA92849
:10015000AD28AE0FAC28AF0A2911B2280030AE008E
:100160000030AF00291DC928273031020319BF28EC
:10017000A00020093105A006A01BC428C8280F3004
:100180003002031CC428C828B00FC728B10A29119F
:10019000CD280030B0000030B100291DD328003038
:1001A000AA000030AB00A9182915A91C2911861A2C
:1001B000DA282911061EDD2829113218E3283130EA
:1001C000B3000030B40032142919FB280030340287
:1001D0000319F128A00020093405A006A01BF62869
:1001E000FA2831303302031CF628FA28B30FF92815
:1001F000B40A2915FF280030B3000030B400291DCF
:1002000016290030360203190C29A00020093605F2
:10021000A006A01B1129152931303502031C112914
:100220001529B50F1429B60A29111A290030B5006D
:100230000030B60029190616291D0612A91829151D
:10024000A91C29110519252929112919B214291DBB
:10025000B2108A012628FF3FFF3FFF3FFF3FFF3FCD
:10026000FF3FFF3FFF3FFF3FFF3FFF3FFF3FFF3F9E
:10027000FF3FFF3FFF3FFF3FFF3FFF3FFF3FFF3F8E
:10028000FF3FFF3FFF3FFF3FFF3FFF3FFF3FFF3F7E
:10029000FF3FFF3FFF3FFF3FFF3FFF3FFF3FFF3F6E
:02400E00503F21
:10420000FF00FF00FF00FF00FF00FF00FF00FF00B6
:10421000FF00FF00FF00FF00FF00FF00FF00FF00A6
:10422000FF00FF00FF00FF00FF00FF00FF00FF0096
:10423000FF00FF00FF00FF00FF00FF00FF00FF0086
:10424000FF00FF00FF00FF00FF00FF00FF00FF0076
:10425000FF00FF00FF00FF00FF00FF00FF00FF0066
:10426000FF00FF00FF00FF00FF00FF00FF00FF0056
:10427000FF00FF00FF00FF00FF00FF00FF00FF0046
:10428000FF00FF00FF00FF00FF00FF00FF00FF0036
:10429000FF00FF00FF00FF00FF00FF00FF00FF0026
:1042A000FF00FF00FF00FF00FF00FF00FF00FF0016
:1042B000FF00FF00FF00FF00FF00FF00FF00FF0006
:1042C000FF00FF00FF00FF00FF00FF00FF00FF00F6
:1042D000FF00FF00FF00FF00FF00FF00FF00FF00E6
:1042E000FF00FF00FF00FF00FF00FF00FF00FF00D6
:1042F000FF00FF00FF00FF00FF00FF00FF00FF00C6
:00000001FF
